:020000001929BC
:10000800FF00030E8301B4000A08B3008A017008D8
:10001800A3007408A2007808A1007C08A0002608A4
:10002800A4002708A5000B1D99282C08F0002D080E
:10003800F1002E08F2002F08F300F00A0319F10A64
:100048000319F20A0319F30A7008AC007108AD002D
:100058007208AE007308AF00F7207008AA00700895
:10006800023A031D5028B20A3208633C03183E289E
:100078006330B2000130AB000A30F4003208F000FF
:10008800AC207008B0000A30F4003208F000AC2050
:100098007808F0007008B1002A08013A031D6D289D
:1000A8002B0803196D28B2033208003A031D5D2896
:1000B800AB010A30F4003208F000AC207008B00040
:1000C8000A30F4003208F000AC207808F00070081C
:1000D800B1002B0803199628051C84280510300840
:1000E800593EF00001300318013EF1007008A600E7
:1000F8007108A700BD208A110A1286008514952868
:1001080085103108593EF00001300318013EF10016
:100118007008A6007108A700BD208A110A1286007F
:1001280005149828051085100B112408A600250829
:10013800A7002308F0002208F4002108F80020088E
:10014800FC0033088A00340E8300FF0E7F0E09007E
:1001580083120313F8010830FC00700DF80D7408C1
:10016800F8020318B928F8070310F00DFC0BB128A2
:0201780008007D
:0E017A008312031327088A002608820008005B
:100188000730831203139F000C3083168500860105
:100198000110811001118115011681128312860147
:0201A80008004D
:0601AA008B168B17080004
:1001B000BD208A110A128000840AA60A0319A70A20
:0801C000F003031DD82808001C
:1001C8000A3083120313F4003508F000AC207008DD
:1001D800B0000A30F4003508F000AC207808F000D0
:0601E8007008B1000800E0
:1001EE0083120313051D0D29851D05292908023AC1
:1001FE0003190229A80A0230A9000C292908013A7C
:10020E0003190A29A80A0130A9000F29A901A8017A
:10021E002808013C03181729A8012908F000080036
:04022E00F0010800D3
:1002320083120313A801A901C420B201AC01AD01CC
:10024200AE01AF01AB01B501E420D5202F08003C7F
:10025200031D35292E08033C031D35292D08933C27
:10026200031D35292C08873C03184229AC01AD0136
:10027200AE01AF012B0803194229B2033208B500BF
:10028200E4203208003C013003180030F0007018FE
:100292004C2985134D2985170D30FC00FB30FD00DC
:1002A200FD0B5129FC0B5129000000002729582978
:1002B2003F3406345B344F3466346D347D34073456
:0402C2007F346F34E2
:02400E0010217F
:00000001FF
